:020000040000FA
:0A0000000000000029EF00F03DD0E1
:0800180090D09EA8FED7AD6E4A
:1000200012000B6A0A6EFF0E0A260B2200D0D8A01F
:100030001200030E096EE60E02D8F5D7096AFE0F0C
:10004000086EE86A095AD8A012000000080600D01D
:10005000F8D7006AB8964F0EAF6EB06A240EAC6E39
:10006000900EAB6E00010F0EC16E070EB46EC69AF5
:10007000C00E926EE00E936EC00E946E956AE80EFE
:10008000966E6ED0F2A409D0F294134A142AD6CFF9
:1000900011F0D7CF12F0817611009EAA19D0060E6A
:1000A000AB1412E1E2CF48F0E1CF47F0492A10EE5D
:1000B0009FF04950E126000EE222AECFE7FF48C094
:1000C000E2FF47C0E1FF1100AE50AE50AB98AB88E5
:1000D000110049504A5C14E04A2AEACF09F0E9CFFE
:1000E00008F000EE9FF04A50E926000EEA22EF5099
:1000F000466E09C0EAFF08C0E9FFD880120004D0AC
:10010000E868466ED8A012001200496A4A6A9D8AC1
:100110009F8AF28EF28C12009D9A00EE9FF0010EE3
:10012000F46EF36AF306000EF45AEE6AF450F3101C
:10013000F9E1496A4A6A9D8A1200F29EE0CF9FFE69
:10014000D8CFA0FEE8CFA1FEF28E0001A192F29ED0
:100150009FCEE0FFA0CED8FFA1CEE8FFF28E100028
:1001600093968A860A0E5DDF93968A9695948C9470
:1001700093908A9094988B9895968C9695988C9855
:10018000949A8B9A959C8C9C959A8C9A95928C9229
:10019000959E8C9E94968B9695908C9094928B9233
:1001A00094948B9496948D9494908B9096908D903B
:1001B00096928D9292988998929A899A929489941B
:1001C000929689969290899092928992206A256857
:1001D00000EE4BF0300EEE68E82EFDD77C6A7B6AAD
:1001E0007E6A7D6A806B7F6A826B816B846B836BB6
:1001F000866B856B886B876B8A6B896B8C6B8B6B63
:100200008E6B8D6B906B8F6B926B916B936B946B12
:10021000956B966B976B986B996B9A6B9B6B9C6BC2
:100220009D6B9E6B2D6A2C6A276A266A2B6A2A6A46
:10023000296A286A6ADF70DFCD6AF294F28A870E33
:10024000D56EB16AA192A092D08EA292B00EB16E7C
:10025000D4EC0DF0D6EC0FF0000EDFDE420EDDDE4A
:10026000590EDBDED6CF11F0D7CF12F032DF46C009
:1002700015F0B10E155C07E3FE0E155C01E301D02D
:10028000176AB2EF05F015AE22D0176A800E155C22
:1002900005E115C017F01868196817D0900E155CA5
:1002A00005E115C017F01A681B680FD0A00E155C89
:1002B00005E115C017F01C681D6807D0B00E155C6D
:1002C00004E115C017F01E681F68B0EF05F0175263
:1002D00004E1B2EF05F0B0EF05F0800E175CD8A492
:1002E000B9D0182803E115C018F0B0D015C019F026
:1002F0001D0E185C0BE1899089924E684D684C6820
:100300004B6826902C9028902A909DD01E0E185C49
:100310000BE1899489965268516850684F6826921B
:100320002C9228922A928FD01F0E185C0BE189988C
:10033000899A566855685468536826942C94289472
:100340002A9481D0200E185C0BE18D908D925A6812
:1003500059685868576826962C9628962A9673D01E
:10036000210E185C0BE18D948B905E685D685C6873
:100370005B6826982C9828982A9865D0220E185CDD
:100380000BE18B928B946268616860685F68269A63
:100390002C9A289A2A9A57D0230E185C0BE18B9638
:1003A0008C906668656864686368269C2C9C289CB1
:1003B0002A9C49D0240E185C0BE18C928C9E6A68B2
:1003C000696868686768269E2C9E289E2A9E3BD096
:1003D000250E185C0BE18C9C8C9A6E686D686C68BD
:1003E0006B6827902D9029902B902DD0260E185CAD
:1003F0000BE18B9A8C987268716870686F682792AD
:100400002D9229922B921FD0270E185C0BE18B980E
:100410008C96766875687468736827942D9429940F
:100420002B9411D0280E185C0BE18C948A907A687A
:1004300079687868776827962D9629962B9603D049
:100440001868B2EF05F01868B2EC0AF0B2EF05F0E8
:10045000B0EF05F0900E175CD8A483EF05F01A28D2
:1004600004E115C01AF081EF05F015C01BF01B5216
:10047000D8A4B2D01D0E1A5C0BE1899089924E6807
:100480004D684C684B6826902C9028902A909DD0FF
:100490001E0E1A5C0BE18994899652685168506867
:1004A0004F6826922C9228922A928FD01F0E1A5CA7
:1004B0000BE18998899A5668556854685368269460
:1004C0002C9428942A9481D0200E1A5C0BE18D90F4
:1004D0008D925A6859685868576826962C962896BF
:1004E0002A9673D0210E1A5C0BE18D948B905E6876
:1004F0005D685C685B6826982C9828982A9865D077
:10050000220E1A5C0BE18B928B94626861686068C2
:100510005F68269A2C9A289A2A9A57D0230E1A5C3A
:100520000BE18B968C906668656864686368269CAE
:100530002C9C289C2A9C49D0240E1A5C0BE18C929E
:100540008C9E6A68696868686768269E2C9E289EEB
:100550002A9E3BD0250E1A5C0BE18C9C8C9A6E680F
:100560006D686C686B6827902D9029902B902DD02A
:10057000260E1A5C0BE18B9A8C9872687168706811
:100580006F6827922D9229922B921FD0270E1A5C0A
:100590000BE18B988C9676687568746873682794FD
:1005A0002D9429942B9411D0280E1A5C0BE18C9475
:1005B0008A907A6879687868776827962D96299660
:1005C0002B9603D01868B2EF05F01A68B2EC0AF067
:1005D000B2EF05F081EF05F020A07CEF05F01D0ED5
:1005E0001A5C34E1268001EE9FF0D8901B34E92696
:1005F000000EEA22EECF2EF0EFCF2FF02E50112476
:10060000026E2F501220036E000E1320046E000E97
:100610001420056E02C04BF003C04CF004C04DF036
:1006200005C04EF08980898293530DE02C800DEE39
:100630009FF0D8909335E926000EEA22EECF7BF0AA
:10064000EFCF7CF001D02C907BEF05F01E0E1A5CF2
:1006500034E1268202EE9FF0D8901B34E926000E8A
:10066000EA22EECF30F0EFCF31F030501124026E9D
:1006700031501220036E000E1320046E000E142061
:10068000056E02C04FF003C050F004C051F005C029
:1006900052F08984898694530DE02C820DEE9FF0F0
:1006A000D8909435E926000EEA22EECF7DF0EFCF08
:1006B0007EF001D02C927BEF05F01F0E1A5C33E127
:1006C00026848988898A03EE9FF0D8901B34E92616
:1006D000000EEA22EECF32F0EFCF33F03250112489
:1006E000026E33501220036E000E1320046E000EB3
:1006F0001420056E02C053F003C054F004C055F03E
:1007000005C056F095530DE02C840DEE9FF0D89067
:100710009535E926000EEA22EECF7FF0EFCF80F08C
:1007200001D02C94E8D1200E1A5C33E126868D800E
:100730008D8204EE9FF0D8901B34E926000EEA2249
:10074000EECF34F0EFCF35F034501124026E355037
:100750001220036E000E1320046E000E1420056E8E
:1007600002C057F003C058F004C059F005C05AF059
:1007700096530DE02C860DEE9FF0D8909635E92625
:10078000000EEA22EECF81F0EFCF82F001D02C965E
:10079000B2D1210E1A5C33E126888D848B8005EE60
:1007A0009FF0D8901B34E926000EEA22EECF36F0F7
:1007B000EFCF37F036501124026E37501220036EFF
:1007C000000E1320046E000E1420056E02C05BF0B4
:1007D00003C05CF004C05DF005C05EF097530DE00F
:1007E0002C880DEE9FF0D8909735E926000EEA226E
:1007F000EECF83F0EFCF84F001D02C987CD1220E85
:100800001A5C33E1268A8B828B8406EE9FF0D890A7
:100810001B34E926000EEA22EECF38F0EFCF39F094
:1008200038501124026E39501220036E000E13202E
:10083000046E000E1420056E02C05FF003C060F06D
:1008400004C061F005C062F098530DE02C8A0DEEF3
:100850009FF0D8909835E926000EEA22EECF85F079
:10086000EFCF86F001D02C9A46D1230E1A5C33E1EB
:10087000268C8C808B8607EE9FF0D8901B34E9265F
:10088000000EEA22EECF3AF0EFCF3BF03A501124BF
:10089000026E3B501220036E000E1320046E000EF9
:1008A0001420056E02C063F003C064F004C065F05C
:1008B00005C066F099530DE02C8C0DEE9FF0D8909A
:1008C0009935E926000EEA22EECF87F0EFCF88F0C7
:1008D00001D02C9C10D1240E1A5C33E1268E8C8220
:1008E0008C8E08EE9FF0D8901B34E926000EEA2289
:1008F000EECF3CF0EFCF3DF03C501124026E3D5066
:100900001220036E000E1320046E000E1420056EDC
:1009100002C067F003C068F004C069F005C06AF067
:100920009A530DE02C8E0DEE9FF0D8909A35E92663
:10093000000EEA22EECF89F0EFCF8AF001D02C9E94
:10094000DAD0250E1A5C33E127808C8C8C8A09EE74
:100950009FF0D8901B34E926000EEA22EECF3EF03D
:10096000EFCF3FF03E501124026E3F501220036E35
:10097000000E1320046E000E1420056E02C06BF0F2
:1009800003C06CF004C06DF005C06EF09B530DE029
:100990002D800DEE9FF0D8909B35E926000EEA22BF
:1009A000EECF8BF0EFCF8CF001D02D90A4D0260E9F
:1009B0001A5C33E127828C888B8A0AEE9FF0D890EC
:1009C0001B34E926000EEA22EECF40F0EFCF41F0D3
:1009D00040501124026E41501220036E000E13206D
:1009E000046E000E1420056E02C06FF003C070F09C
:1009F00004C071F005C072F09C530DE02D820DEE25
:100A00009FF0D8909C35E926000EEA22EECF8DF0BB
:100A1000EFCF8EF001D02D926ED0270E1A5C33E10D
:100A200027848B888C860BEE9FF0D8901B34E926A8
:100A3000000EEA22EECF42F0EFCF43F042501124F5
:100A4000026E43501220036E000E1320046E000E3F
:100A50001420056E02C073F003C074F004C075F07A
:100A600005C076F09D530DE02D840DEE9FF0D890DB
:100A70009D35E926000EEA22EECF8FF0EFCF90F001
:100A800001D02D9438D0280E1A5C33E127868C844F
:100A90008A800CEE9FF0D8901B34E926000EEA22E3
:100AA000EECF44F0EFCF45F044501124026E455094
:100AB0001220036E000E1320046E000E1420056E2B
:100AC00002C077F003C078F004C079F005C07AF076
:100AD0009E530DE02D860DEE9FF0D8909E35E926B1
:100AE000000EEA22EECF91F0EFCF92F001D02D96DA
:100AF00002D01A6837D002D01A6834D01A68B2EC23
:100B00000AF030D02DD0A00E175C1DE11C2803E1A7
:100B100015C01CF016D015C01DF020A012D01D0E5F
:100B20001C5C000ED8B0010E106E290E1C5C02E396
:100B3000000E01D0010E101604E0ECEC0AF0B2EC4D
:100B40000AF010D00DD0B00E175C0AE11E2803E1A8
:100B500015C01EF004D015C01FF06DEC0CF002D0D3
:100B6000B2EC0AF00C0E255CD8B0A9EF0AF02150C7
:100B7000115C225012582350135824501458D8A0F6
:100B80009CEF0AF0248E2552D8A464D02CB007D054
:100B90004E684D684C684B682690899259D02AA0BF
:100BA00019D026802E501124026E2F501220036E71
:100BB000000E1320046E000E1420056E02C04BF0D0
:100BC00003C04CF004C04DF005C04EF0898289800E
:100BD0002A903ED028A023D089900DEE9FF0D89087
:100BE0009335E926000EEA22EECF06F0EFCF07F0AC
:100BF00006501124026E07501220036E000E1320BF
:100C0000046E000E1420056E02C04BF003C04CF0C1
:100C100004C04DF005C04EF028902A8019D026A0BF
:100C200017D089927B501124026E7C501220036EE3
:100C3000000E1320046E000E1420056E02C04BF04F
:100C400003C04CF004C04DF005C04EF02880269043
:100C50009BEF0AF0010E255CD8A464D02CB207D01B
:100C600089965268516850684F68269259D02AA2D6
:100C700019D0268230501124026E31501220036E9A
:100C8000000E1320046E000E1420056E02C04FF0FB
:100C900003C050F004C051F005C052F08986898429
:100CA0002A923ED028A223D089940DEE9FF0D890AE
:100CB0009435E926000EEA22EECF06F0EFCF07F0DA
:100CC00006501124026E07501220036E000E1320EE
:100CD000046E000E1420056E02C04FF003C050F0E9
:100CE00004C051F005C052F028922A8219D026A2E1
:100CF00017D089967D501124026E7E501220036E0B
:100D0000000E1320046E000E1420056E02C04FF07A
:100D100003C050F004C051F005C052F02882269262
:100D20009BEF0AF0020E255CD8A464D02CB407D047
:100D3000899A5668556854685368269459D02AA4ED
:100D400019D0268432501124026E33501220036EC3
:100D5000000E1320046E000E1420056E02C053F026
:100D600003C054F004C055F005C056F0898A898844
:100D70002A943ED028A423D089980DEE9FF0D890D5
:100D80009535E926000EEA22EECF06F0EFCF07F008
:100D900006501124026E07501220036E000E13201D
:100DA000046E000E1420056E02C053F003C054F010
:100DB00004C055F005C056F028942A8419D026A402
:100DC00017D0899A7F501124026E80511220036E31
:100DD000000E1320046E000E1420056E02C053F0A6
:100DE00003C054F004C055F005C056F02884269482
:100DF0009BEF0AF0030E255CD8A464D02CB607D074
:100E00008D925A68596858685768269659D02AA60C
:100E100019D0268634501124026E35501220036EEC
:100E2000000E1320046E000E1420056E02C057F051
:100E300003C058F004C059F005C05AF08D828D806F
:100E40002A963ED028A623D08D900DEE9FF0D89004
:100E50009635E926000EEA22EECF06F0EFCF07F036
:100E600006501124026E07501220036E000E13204C
:100E7000046E000E1420056E02C057F003C058F037
:100E800004C059F005C05AF028962A8619D026A623
:100E900017D08D9281511124026E82511220036E5F
:100EA000000E1320046E000E1420056E02C057F0D1
:100EB00003C058F004C059F005C05AF028862696A1
:100EC0009BEF0AF0040E255CD8A464D02CB807D0A0
:100ED0008B905E685D685C685B68269859D02AA82C
:100EE00019D0268836501124026E37501220036E16
:100EF000000E1320046E000E1420056E02C05BF07D
:100F000003C05CF004C05DF005C05EF08B808D8492
:100F10002A983ED028A823D08D940DEE9FF0D8902B
:100F20009735E926000EEA22EECF06F0EFCF07F064
:100F300006501124026E07501220036E000E13207B
:100F4000046E000E1420056E02C05BF003C05CF05E
:100F500004C05DF005C05EF028982A8819D026A844
:100F600017D08B9083511124026E84511220036E8E
:100F7000000E1320046E000E1420056E02C05BF0FC
:100F800003C05CF004C05DF005C05EF028882698C0
:100F90009BEF0AF0050E255CD8A464D02CBA07D0CC
:100FA0008B946268616860685F68269A59D02AAA43
:100FB00019D0268A38501124026E39501220036E3F
:100FC000000E1320046E000E1420056E02C05FF0A8
:100FD00003C060F004C061F005C062F08B848B82B6
:100FE0002A9A3ED028AA23D08B920DEE9FF0D8905B
:100FF0009835E926000EEA22EECF06F0EFCF07F093
:1010000006501124026E07501220036E000E1320AA
:10101000046E000E1420056E02C05FF003C060F085
:1010200004C061F005C062F0289A2A8A19D026AA65
:1010300017D08B9485511124026E86511220036EB5
:10104000000E1320046E000E1420056E02C05FF027
:1010500003C060F004C061F005C062F0288A269ADF
:101060009BEF0AF0060E255CD8A463D02CBC07D0F9
:101070008C906668656864686368269C59D02AAC61
:1010800019D0268C3A501124026E3B501220036E68
:10109000000E1320046E000E1420056E02C063F0D3
:1010A00003C064F004C065F005C066F08C808B86D8
:1010B0002A9C3ED028AC23D08B960DEE9FF0D89082
:1010C0009935E926000EEA22EECF06F0EFCF07F0C1
:1010D00006501124026E07501220036E000E1320DA
:1010E000046E000E1420056E02C063F003C064F0AD
:1010F00004C065F005C066F0289C2A8C19D026AC87
:1011000017D08C9087511124026E88511220036EE3
:10111000000E1320046E000E1420056E02C063F052
:1011200003C064F004C065F005C066F0288C269CFE
:1011300002D2070E255CD8A463D02CBE07D08C9EAB
:101140006A68696868686768269E59D02AAE19D0AF
:10115000268E3C501124026E3D501220036E000E6C
:101160001320046E000E1420056E02C067F003C049
:1011700068F004C069F005C06AF08C8E8C822A9EEB
:101180003ED028AE23D08C920DEE9FF0D8909A35A9
:10119000E926000EEA22EECF06F0EFCF07F0065068
:1011A0001124026E07501220036E000E1320046EED
:1011B000000E1420056E02C067F003C068F004C082
:1011C00069F005C06AF0289E2A8E19D026AE17D085
:1011D0008C9E89511124026E8A511220036E000EDA
:1011E0001320046E000E1420056E02C067F003C0C9
:1011F00068F004C069F005C06AF0288E269E9BD175
:10120000080E255CD8A463D02DB007D08C9A6E68E8
:101210006D686C686B68279059D02BA019D0278017
:101220003E501124026E3F501220036E000E132018
:10123000046E000E1420056E02C06BF003C06CF04B
:1012400004C06DF005C06EF08C8A8C8C2B903ED063
:1012500029A023D08C9C0DEE9FF0D8909B35E926D9
:10126000000EEA22EECF06F0EFCF07F00650112471
:10127000026E07501220036E000E1320046E000E43
:101280001420056E02C06BF003C06CF004C06DF05A
:1012900005C06EF029902B8019D027A017D08C9A0A
:1012A0008B511124026E8C511220036E000E1320FC
:1012B000046E000E1420056E02C06BF003C06CF0CB
:1012C00004C06DF005C06EF02980279034D1090E5E
:1012D000255CD8A463D02DB207D08B9A7268716850
:1012E00070686F68279259D02BA219D0278240507E
:1012F0001124026E41501220036E000E1320046E62
:10130000000E1420056E02C06FF003C070F004C020
:1013100071F005C072F08B8A8C882B923ED029A286
:1013200023D08C980DEE9FF0D8909C35E926000EC6
:10133000EA22EECF06F0EFCF07F006501124026E3E
:1013400007501220036E000E1320046E000E1420AE
:10135000056E02C06FF003C070F004C071F005C0EC
:1013600072F029922B8219D027A217D08B9A8D5117
:101370001124026E8E511220036E000E1320046E93
:10138000000E1420056E02C06FF003C070F004C0A0
:1013900071F005C072F029822792CDD00A0E255C2B
:1013A000D8A463D02DB407D08C967668756874681D
:1013B0007368279459D02BA419D027844250112444
:1013C000026E43501220036E000E1320046E000EB6
:1013D0001420056E02C073F003C074F004C075F0F1
:1013E00005C076F08C868B882B943ED029A423D020
:1013F0008B980DEE9FF0D8909D35E926000EEA22DD
:10140000EECF06F0EFCF07F006501124026E075022
:101410001220036E000E1320046E000E1420056EC1
:1014200002C073F003C074F004C075F005C076F01C
:1014300029942B8419D027A417D08C968F5111246E
:10144000026E90511220036E000E1320046E000EE7
:101450001420056E02C073F003C074F004C075F070
:1014600005C076F02984279466D00B0E255CD8A49D
:1014700062D02DB607D08A907A68796878687768E4
:10148000279659D02BA619D0278644501124026ED6
:1014900045501220036E000E1320046E000E14201F
:1014A000056E02C077F003C078F004C079F005C083
:1014B0007AF08A808C842B963ED029A623D08C94F7
:1014C0000DEE9FF0D8909E35E926000EEA22EECF71
:1014D00006F0EFCF07F006501124026E07501220DD
:1014E000036E000E1320046E000E1420056E02C061
:1014F00077F003C078F004C079F005C07AF029963F
:101500002B8619D027A617D08A9091511124026EEC
:1015100092511220036E000E1320046E000E142050
:10152000056E02C077F003C078F004C079F005C002
:101530007AF02986279616D814AE0AD0146A136A50
:10154000126A116A00EE4BF0300EEE68E82EFDD7FD
:1015500006D014AE04D0146A136A126A116A817834
:1015600032EF01F02568248E166A0C0E165C33E209
:10157000D8901634E96EEA6AEA36E936EA364B0E56
:10158000E926000EEA22EFCF02F0ECCF03F0ECCF19
:1015900004F0ECCF05F02150025C22500358235098
:1015A00004582450055815E2D8901634E96EEA6ABA
:1015B000EA36E936EA364B0EE926000EEA22EFCF8C
:1015C00021F0ECCF22F0ECCF23F0ECCF24F016C0CA
:1015D00025F0162ACAE312001D0E1C5C1DE11DC079
:1015E00093F093530CE00DEE9FF0D8909335E926DD
:1015F000000EEA22EECF7BF0EFCF7CF00CD07C6ABD
:101600007B6A2C90269028902A904E684D684C68F2
:101610004B68899089925FD11E0E1C5C1DE11DC034
:1016200094F094530CE00DEE9FF0D8909435E92699
:10163000000EEA22EECF7DF0EFCF7EF00CD07E6A76
:101640007D6A2C92269228922A925268516850689C
:101650004F68899489963FD11F0E1C5C1DE11DC007
:1016600095F095530CE00DEE9FF0D8909535E92656
:10167000000EEA22EECF7FF0EFCF80F00CD0806B2F
:101680007F6A2C94269428942A9456685568546846
:1016900053688998899A1FD1200E1C5C1DE11DC0DA
:1016A00096F096530CE00DEE9FF0D8909635E92613
:1016B000000EEA22EECF81F0EFCF82F00CD0826BE9
:1016C000816B2C96269628962A965A6859685868EF
:1016D00057688D908D92FFD0210E1C5C1DE11DC0BE
:1016E00097F097530CE00DEE9FF0D8909735E926D0
:1016F000000EEA22EECF83F0EFCF84F00CD0846BA3
:10170000836B2C98269828982A985E685D685C6898
:101710005B688D948B90DFD0220E1C5C1DE11DC098
:1017200098F098530CE00DEE9FF0D8909835E9268C
:10173000000EEA22EECF85F0EFCF86F00CD0866B5C
:10174000856B2C9A269A289A2A9A62686168606842
:101750005F688B928B94BFD0230E1C5C1DE11DC073
:1017600099F099530CE00DEE9FF0D8909935E92649
:10177000000EEA22EECF87F0EFCF88F00CD0886B16
:10178000876B2C9C269C289C2A9C666865686468EC
:1017900063688B968C909FD0240E1C5C1DE11DC04D
:1017A0009AF09A530CE00DEE9FF0D8909A35E92606
:1017B000000EEA22EECF89F0EFCF8AF00CD08A6BD0
:1017C000896B2C9E269E289E2A9E6A686968686896
:1017D00067688C928C9E7FD0250E1C5C1DE11DC01D
:1017E0009BF09B530CE00DEE9FF0D8909B35E926C3
:1017F000000EEA22EECF8BF0EFCF8CF00CD08C6B8A
:101800008B6B2D90279029902B906E686D686C687B
:101810006B688C9C8C9A5FD0260E1C5C1DE11DC0F1
:101820009CF09C530CE00DEE9FF0D8909C35E9267F
:10183000000EEA22EECF8DF0EFCF8EF00CD08E6B43
:101840008D6B2D92279229922B9272687168706825
:101850006F688C988B9A3FD0270E1C5C1DE11DC0D1
:101860009DF09D530CE00DEE9FF0D8909D35E9263C
:10187000000EEA22EECF8FF0EFCF90F00CD0906BFD
:101880008F6B2D94279429942B94766875687468CF
:1018900073688B988C961FD0280E1C5C1CE11DC0B1
:1018A0009EF09E530CE00DEE9FF0D8909E35E926F9
:1018B000000EEA22EECF91F0EFCF92F00CD0926BB7
:1018C000916B2D96279629962B967A687968786879
:1018D00077688C948A901C6812001E0E1E5CD8A437
:1018E000EDD01F52D8A44BD02D6A2C6A7C6A7B6A3B
:1018F000936B7E6A7D6A946B806B7F6A956B826B5B
:10190000816B966B846B836B976B866B856B986B27
:10191000886B876B996B8A6B896B9A6B8C6B8B6B03
:101920009B6B8E6B8D6B9C6B906B8F6B9D6B926BBF
:10193000916B9E6B276A266A296A286A2B6A2A6A33
:1019400000EE4BF0300EEE68E82EFDD78C948B98AD
:101950008C988C9C8C928B968B928D948D90899880
:10196000899489908A908C968B9A8C9A8C9E8C9074
:101970008B948B908D92899A899689929CD01FC066
:1019800093F00DEE9FF0D8901F34E926000EEA2266
:10199000EECF7BF0EFCF7CF01FC094F00DEE9FF008
:1019A000D8901F34E926000EEA22EECF7DF0EFCF6B
:1019B0007EF01FC095F00DEE9FF0D8901F34E92601
:1019C000000EEA22EECF7FF0EFCF80F01FC096F03E
:1019D0000DEE9FF0D8901F34E926000EEA22EECFDC
:1019E00081F0EFCF82F01FC097F00DEE9FF0D890FE
:1019F0001F34E926000EEA22EECF83F0EFCF84F009
:101A00001FC098F00DEE9FF0D8901F34E926000E0D
:101A1000EA22EECF85F0EFCF86F01FC099F00DEEF1
:101A20009FF0D8901F34E926000EEA22EECF87F00F
:101A3000EFCF88F01FC09AF00DEE9FF0D8901F34C2
:101A4000E926000EEA22EECF89F0EFCF8AF01FC020
:101A50009BF00DEE9FF0D8901F34E926000EEA228D
:101A6000EECF8BF0EFCF8CF01FC09CF00DEE9FF00F
:101A7000D8901F34E926000EEA22EECF8DF0EFCF8A
:101A80008EF01FC09DF00DEE9FF0D8901F34E92618
:101A9000000EEA22EECF8FF0EFCF90F01FC09EF045
:101AA0000DEE9FF0D8901F34E926000EEA22EECF0B
:101AB00091F0EFCF92F0B2EC0AF02ED0420E1E5C05
:101AC00008E11F5203E1209029D802D020808A82A9
:101AD00023D07B0E1E5C20E100EE4BF0300EEE6852
:101AE000E82EFDD78C948B988C988C9C8C928B963E
:101AF0008B928D948D908998899489908A908C96F8
:101B00008B9A8C9A8C9E8C908B948B908D92899AC8
:101B10008996899220B08A821E68120000EE4BF0EE
:101B2000300EEE68E82EFDD78C948B988C988C9CA8
:101B30008C928B968B928D948D90899889948990B4
:101B40008A908C968B9A8C9A8C9E8C908B948B908E
:101B50008D92899A899689928A922D6A2C6A7C6ADA
:101B60007B6A936B7E6A7D6A946B806B7F6A956BF0
:101B7000826B816B966B846B836B976B866B856BCB
:101B8000986B886B876B996B8A6B896B9A6B8C6B84
:101B90008B6B9B6B8E6B8D6B9C6B906B8F6B9D6B54
:101BA000926B916B9E6B12000D01A0699F69270ECD
:101BB000A26F100EA16F250EA46FCE0EA36F250E7F
:101BC000A66F300EA56F240EA86F960EA76F230E7A
:101BD000AA6FFE0EA96F230EAC6F680EAB6F220EBC
:101BE000AE6FD50EAD6F220EB06F440EAF6F210EEB
:101BF000B26FB60EB16F210EB46F290EB36F200E07
:101C0000B66FA00EB56F200EB86F180EB76F1F0E0F
:101C1000BA6F920EB96F1F0EBC6F0F0EBB6F1E0E08
:101C2000BE6F8E0EBD6F1E0EC06F0F0EBF6F1D0EEE
:101C3000C26F920EC16F1D0EC46F170EC36F1C0EC4
:101C4000C66F9E0EC56F1C0EC86F270EC76F1B0E8A
:101C5000CA6FB20EC96F1B0ECC6F3F0ECB6F1A0E40
:101C6000CE6FCE0ECD6F1A0ED06F5E0ECF6F190EE7
:101C7000D26FF10ED16F190ED46F850ED36F190E7E
:101C8000D66F1B0ED56F180ED86FB20ED76F180E09
:101C9000DA6F4C0ED96F170EDC6FE70EDB6F170E85
:101CA000DE6F830EDD6F170EE06F210EDF6F160EF5
:101CB000E26FC10EE16F160EE46F630EE36F160E56
:101CC000E66F060EE56F150EE86FAA0EE76F150EAC
:101CD000EA6F500EE96F140EEC6FF70EEB6F140EF7
:101CE000EE6FA00EED6F140EF06F4A0EEF6F130E35
:101CF000F26FF60EF16F130EF46FA30EF36F130E67
:101D0000F66F510EF56F130EF86F010EF76F120E8E
:101D1000FA6FB20EF96F120EFC6F640EFB6F120EAB
:101D2000FE6F180EFD6F0E01110E006F0D01CD0E2E
:101D3000FF6F0E01110E026F830E016F110E046F03
:101D40003A0E036F100E066FF20E056F100E086F3D
:101D5000AC0E076F100E0A6F660E096F100E0C6F37
:101D6000220E0B6F0F0E0E6FDF0E0D6F0F0E106F2A
:101D70009D0E0F6F0F0E126F5C0E116F0F0E146F12
:101D80001C0E136F0E0E166FDE0E156F0E0E186FF3
:101D9000A00E176F0E0E1A6F630E196F0E0E1C6FCA
:101DA000270E1B6F0D0E1E6FEC0E1D6F0D0E206F9C
:101DB000B20E1F6F0D0E226F7A0E216F0D0E246F63
:101DC000410E236F0D0E266F0A0E256F0C0E286F25
:101DD000D40E276F0C0E2A6F9F0E296F0C0E2C6FDE
:101DE0006A0E2B6F0C0E2E6F370E2D6F0C0E306F90
:101DF000040E2F6F0B0E326FD20E316F0B0E346F3D
:101E0000A10E336F0B0E366F700E356F0B0E386FE1
:101E1000410E376F0B0E3A6F120E396F0A0E3C6F80
:101E2000E40E3B6F0A0E3E6FB70E3D6F0A0E406F19
:101E30008A0E3F6F0A0E426F5E0E416F0A0E446FAC
:101E4000330E436F0A0E466F090E456F486FDF0E63
:101E5000476F090E4A6FB60E496F090E4C6F8E0E12
:101E60004B6F090E4E6F660E4D6F090E506F3F0E91
:101E70004F6F090E526F190E516F080E546FF30E0B
:101E8000536F080E566FCD0E556F080E586FA90E82
:101E9000576F080E5A6F850E596F080E5C6F610EF2
:101EA0005B6F080E5E6F3F0E5D6F080E606F1C0E5D
:101EB0005F6F070E626FFB0E616F070E646FD90EC6
:101EC000636F070E666FB90E656F070E686F990E28
:101ED000676F070E6A6F790E696F070E6C6F5A0E87
:101EE0006B6F070E6E6F3B0E6D6F070E706F1D0EE2
:101EF0006F6F070E726F716B060E746FE30E736F68
:101F0000060E766FC60E756F060E786FAA0E776F87
:101F1000060E7A6F8E0E796F060E7C6F730E7B6FD6
:101F2000060E7E6F580E7D6F060E806F3E0E7F6F21
:101F3000060E826F240E816F060E846F0A0E836F69
:101F4000050E866FF10E856F050E886FD80E876FB0
:101F5000050E8A6FC00E896F050E8C6FA80E8B6FF1
:101F6000050E8E6F910E8D6F050E906F7A0E8F6F2E
:101F7000050E926F630E916F050E946F4C0E936F6A
:101F8000050E966F360E956F050E986F210E976FA2
:101F9000050E9A6F0B0E996F040E9C6FF60E9B6FD9
:101FA000040E9E6FE20E9D6F00011200166A800EF5
:101FB000165CD8B00CD10F6A960E16240E6ED8B0EF
:101FC0000F2A16500E24026E000E0F20036E01EE33
:101FD0009FF0D8901634E926000EEA2202C0EEFFE8
:101FE00003C0EFFF01EE9FF0D8901634E926000EF3
:101FF000EA22EECF02F0EFCF03F002EE9FF0D8908E
:102000001634E926000EEA2202C0EEFF03C0EFFFFD
:1020100001EE9FF0D8901634E926000EEA22EECFAA
:1020200002F0EFCF03F003EE9FF0D8901634E926CC
:10203000000EEA2202C0EEFF03C0EFFF01EE9FF0A8
:10204000D8901634E926000EEA22EECF02F0EFCF48
:1020500003F004EE9FF0D8901634E926000EEA2231
:1020600002C0EEFF03C0EFFF01EE9FF0D8901634E0
:10207000E926000EEA22EECF02F0EFCF03F005EEE4
:102080009FF0D8901634E926000EEA2202C0EEFF37
:1020900003C0EFFF01EE9FF0D8901634E926000E42
:1020A000EA22EECF02F0EFCF03F006EE9FF0D890D9
:1020B0001634E926000EEA2202C0EEFF03C0EFFF4D
:1020C00001EE9FF0D8901634E926000EEA22EECFFA
:1020D00002F0EFCF03F007EE9FF0D8901634E92618
:1020E000000EEA2202C0EEFF03C0EFFF01EE9FF0F8
:1020F000D8901634E926000EEA22EECF02F0EFCF98
:1021000003F008EE9FF0D8901634E926000EEA227C
:1021100002C0EEFF03C0EFFF01EE9FF0D89016342F
:10212000E926000EEA22EECF02F0EFCF03F009EE2F
:102130009FF0D8901634E926000EEA2202C0EEFF86
:1021400003C0EFFF01EE9FF0D8901634E926000E91
:10215000EA22EECF02F0EFCF03F00AEE9FF0D89024
:102160001634E926000EEA2202C0EEFF03C0EFFF9C
:1021700001EE9FF0D8901634E926000EEA22EECF49
:1021800002F0EFCF03F00BEE9FF0D8901634E92663
:10219000000EEA2202C0EEFF03C0EFFF01EE9FF047
:1021A000D8901634E926000EEA22EECF02F0EFCFE7
:1021B00003F00CEE9FF0D8901634E926000EEA22C8
:1021C00002C0EEFF03C0EFFF162AD8A0F0D612001F
:0221D000FFD737
:020000040030CA
:0300010006160ED2
:020005008580F4
:060008000FC00FE00F40E5
:00000001FF
